:100000000C9482000C9494000C9494000C94940032
:100010000C9494000C9494000C9494000C94940010
:100020000C9494000C9494000C9494000C94940000
:100030000C9494000C9494000C9494000C949400F0
:100040000C9473080C9494000C9494000C949400F9
:100050000C9494000C9494000C9494000C949400D0
:100060000C9494000C9494004D025C068402BA0235
:100070002E03F10327045D047E04AC045C067405C2
:10008000F0054903B10350035B0371037C0385034F
:1000900091039A03A603C8042E05D204DA04EE04E1
:1000A000F60402050B0517052005000000080002F4
:1000B000010000030407000000000000000001022E
:1000C00004081020408001020408102001020408E6
:1000D00010200404040404040404020202020202C4
:1000E000030303030303000000002300260029008C
:1000F00000000000250028002B0000000000240064
:1001000027002A0011241FBECFEFD8E0DEBFCDBFED
:1001100022E0A0E0B1E001C01D92A937B207E1F7EB
:100120000E9464080C94CB090C9400008091540246
:10013000811104C08CE392E00C94B2060895809182
:100140006202811104C08CE392E00C94AE06089523
:10015000EF920F931F93E02E89019A01AB01BC012E
:1001600088E091E00E942C071F910F91EF90089575
:1001700088E091E00C9479070F931F934FE950E0CA
:1001800063E070E082E692E00E94FE0646E950E0FD
:1001900062E070E084E592E00E94FE0661E088E0A3
:1001A0000E942D0961E08CE00E942D0961E089E048
:1001B0000E942D0961E084E00E942D0961E085E044
:1001C0000E942D0961E086E00E942D090EE816E0EC
:1001D00024E130E040E050E060E171E088E091E04F
:1001E0000E94AD078CE392E00E949F018CE392E0B5
:1001F0001F910F910C94BB01CF92DF92EF92FF926F
:100200000E94BD086B017C0182E692E00E94B60666
:1002100084E592E00E94B6064091040150910501E8
:100220006091060170910701809100019091010198
:10023000A0910201B0910301452B462B472B59F0A9
:10024000AC01BD01465F5F4F6F4F7F4FC416D506AF
:10025000E606F70648F1B701A601481B590B6A0BE1
:100260007B0B88E091E00E94DA078CE392E00E9429
:10027000E601C0920001D0920101E0920201F092E9
:1002800003018091040190910501A0910601B091B4
:1002900007010196A11DB11D8093040190930501F2
:1002A000A0930601B0930701FF90EF90DF90CF90ED
:1002B0000895CF93DF93EC010E949C06882311F0F0
:1002C00061E001C060E089E00E946609CE010E9401
:1002D0009F06882311F061E001C060E08CE00E947D
:1002E0006609CE010E94A206882311F061E001C0D8
:1002F00060E088E00E946609CE010E94A80688237B
:1003000011F061E001C060E084E00E946609CE0166
:100310000E94AB06882311F061E001C060E085E037
:100320000E946609CE010E94A506882311F061E0B3
:1003300001C060E086E0DF91CF910C946609FC017A
:100340008EE090E09183808313821282128613865E
:100350001486158616861786108A118A128A138AC1
:10036000148A158A168A178A1482158216821782B1
:100370001086118608950F93CF93DF93EC01BC0193
:10038000695E7F4F01E028EC30E040E050E00E94E1
:10039000A8001C821E821D8218861986BE016B5E13
:1003A0007F4F00E024EF31E040E050E0CE010E94BA
:1003B000A80081E08D838F838CE090E0998388830F
:1003C0001B821A82DF91CF910F9108952F923F9255
:1003D0004F925F926F927F928F929F92AF92BF9255
:1003E000CF92DF92EF92FF920F93CF93DF93CDB72F
:1003F000DEB72C970FB6F894DEBF0FBECDBF9C873B
:100400008B87DC0113961C921E9212972EE0622EAF
:10041000712C5696BA87A9875C01B5E1AB0EB11C69
:10042000FC017496FA83E9831C01F3E12F0E311C61
:1004300042969C838B83AB85BC855196BE83AD83EE
:10044000EB85FC857096F887EF834B845C84FFE036
:100450004F0E511C8B849C848EE0880E911CEB8483
:10046000FC849CE0E90EF11CCB84DC84ADE0CA0E78
:10047000D11CEB85FC8582819381892B09F028C4EE
:10048000AB85BC85ED91FC913197ED30F10508F01D
:1004900013C4EC5CFF4F0C94C509EB85FC85878980
:1004A000882319F0CF010E945901AB85BC851B96AA
:1004B0008C911B978111E2C0AB85BC851A968C91FB
:1004C0001A97882309F4F8C311967C926E921396BA
:1004D0001C921E92129700E028E53BE140E050E0BC
:1004E000B701CD010E94A80024EF31E040E050E0C8
:1004F000B6018B859C850E94A80081E0EB85FC8578
:10050000878383E090E0D4C3AB85BC8557968C91FC
:100510005797882319F0CD010E945901EB85FC857E
:100520008385811129C2AB85BC851C968C911C9753
:10053000811136C0EB85FC858585882309F4BCC311
:100540007182608213821282B601CF010E94B800CC
:1005500000E024EF31E040E050E0B4018B859C8561
:100560000E94A800AB85BC8517961C92179784E063
:1005700090E00AC3EB85FC858789882319F0CF01B9
:100580000E945901AB85BC851B968C911B978111EC
:1005900075C0AB85BC851C968C911C978823E9F1AE
:1005A0008D919C918330910571F00497B1F4AB85E6
:1005B000BC8511967C926E9213961C921E92129795
:1005C000B401CD0108C0EB85FC8571826082138285
:1005D0001282B601CF010E94B800B7018B859C85BD
:1005E0000E94B800EB85FC85178200E020ED37E023
:1005F00040E050E0B201CF010E94A800AB85BC856D
:1006000014961C92149781E015968C931597169664
:100610001C92169785E090E0B7C2EB85FC85868535
:10062000882309F449C37182608213821282B40163
:10063000CF010E94B80000E024EF31E040E050E03C
:10064000B6018B859C850E94A80081E0AB85BC85A6
:1006500017968C93179783E090E096C2EB85FC8504
:100660008789882319F0CF010E945901AB85BC8589
:100670001B968C911B97882309F48CC0ED91FC91FB
:100680003197EA30F10508F06CC0EF5BFF4F0C9436
:10069000C509EB85FC85718260821382128261C07C
:1006A000AB85BC8511967C926E9213961C921E921D
:1006B0001297B6010AC0AB85BC8511967C926E92EA
:1006C00013961C921E921297B401CD010E94B8009D
:1006D000B7018B859C850E94B800EB85FC8517824D
:1006E00040C0AB85BC8511967C926E9213961C928D
:1006F0001E921297B20128C0EB85FC857182608240
:10070000138212826F81788529C0AB85BC851196D2
:100710007C926E9213961C921E9212976D817E812E
:1007200013C0EB85FC8571826082138212826B811B
:100730007C8114C0AB85BC8511967C926E92139619
:100740001C921E921297B101CD0109C0EB85FC8568
:10075000718260821382128269817A81CF010E9444
:10076000B800AB85BC8514961C92149716961C9203
:10077000169715961C92159718961C92189719960D
:100780001C92199700E024EF31E040E050E0B50101
:10079000CD0185C2AB85BC851F968C911F978823A0
:1007A00009F48AC211967C926E9213961C921E9244
:1007B0001297B201CD010E94B80000E020ED37E0B1
:1007C00040E050E06F8178858B859C850E94A80071
:1007D00081E0EB85FC8584831582168286E090E0BB
:1007E00067C2AB85BC8557968C915797882319F0C3
:1007F000CD010E945901EB85FC8583858111BCC028
:10080000AB85BC8550968C915097882309F454C2CF
:1008100011967C926E9213961C921E9212976F8183
:100820007885CD010E94B80000E028E53BE140E07A
:1008300050E06D817E818B859C850E94A800EB85B0
:10084000FC85108681E0818787E090E031C2AB852E
:10085000BC8557968C915797882319F0CD010E943B
:100860005901EB85FC858385811186C0AB85BC85EC
:1008700051968C915197882309F41EC211967C924F
:100880006E9213961C921E9212976D817E81CD01FD
:100890000E94B80000E028E833E140E050E06B81BE
:1008A0007C818B859C850E94A80081E0EB85FC857E
:1008B0008087118688E090E0FBC1AB85BC855796A8
:1008C0008C915797882319F0CD010E945901EB852F
:1008D000FC858385811150C0AB85BC8552968C9177
:1008E0005297882309F4E8C111967C926E92139670
:1008F0001C921E9212976B817C81E0C0AB85BC85F7
:1009000057968C915797882319F0CD010E94590171
:10091000EB85FC85838581112FC0AB85BC85539603
:100920008C915397882309F4C7C111967C926E92DB
:1009300013961C921E921297B101CD010E94B8002D
:10094000EB85FC851482158281E086838087118681
:10095000178281E090E0ACC1AB85BC8557968C9145
:100960005797882319F0CD010E945901EB85FC852A
:100970008385882309F491C00190F081E02D31979F
:10098000EA30F10508F06AC0E55BFF4F0C94C50939
:10099000AB85BC8511967C926E9213961C921E922A
:1009A00012975CC0EB85FC85718260821382128293
:1009B000B60107C0EB85FC857182608213821282CA
:1009C000B401CF010E94B800B7018B859C850E94BD
:1009D000B800AB85BC8517961C9240C0EB85FC85A2
:1009E0007182608213821282B20128C0AB85BC85FD
:1009F00011967C926E9213961C921E9212976F81A2
:100A0000788529C0EB85FC85718260821382128211
:100A10006D817E8113C0AB85BC8511967C926E92F0
:100A200013961C921E9212976B817C8114C0EB85E9
:100A3000FC857182608213821282B101CF010CC0E9
:100A4000AB85BC8511967C926E9213961C921E9279
:100A5000129769817A81CD010E94B800EB85FC85EF
:100A60001482168215821086118600E024EF31E090
:100A700040E050E0B501CF010E94A80081E0AB85C5
:100A8000BC8515968C93159717968C931797ECE069
:100A9000F0E01196FC93EE937AC0AB85BC8554963A
:100AA0008C915497882309F407C111967C926E9219
:100AB00013961C921E92129769817A81CD010E9431
:100AC000B80000E020ED37E040E050E0B1018B8558
:100AD0009C850E94A80081E0EB85FC85848385834A
:100AE000168289E090E0E4C0AB85BC8557968C9176
:100AF0005797882319F0CD010E945901EB85FC8599
:100B00008385882309F448C0808191818C309105C8
:100B100061F00D97B9F4EB85FC85718260821382D8
:100B2000128269857A85CF010BC0AB85BC85119691
:100B30007C926E9213961C921E921297B501CD0173
:100B40000E94B80000E020E137E240E050E0698117
:100B50007A818B859C850E94A80081E0AB85BC854D
:100B600014968C93149715961C92159716961C92B2
:100B7000169718968C93189719961C921997179692
:100B80001C9217978AE090E011969C938E9313968F
:100B90001C921E92129790C0EB85FC858589882354
:100BA00009F48AC07182608213821282B501CF017A
:100BB0000E94B80000E024EF31E040E050E0698599
:100BC0007A858B859C850E94A800AB85BC8515968F
:100BD0001C92159717961C9217978DE090E0D4CF32
:100BE000EB85FC858789882319F0CF010E94590184
:100BF000AB85BC851B968C911B978823A9F18D91A1
:100C00009C918C30910579F00D97B9F4AB85BC853A
:100C100011967C926E9213961C921E921297698581
:100C20007A85CD0108C0EB85FC85718260821382D4
:100C30001282B501CF010E94B80000E020E137E246
:100C400040E050E069817A818B859C850E94A800F4
:100C500081E0EB85FC85848315821682808711866E
:100C600017828AE090E024C0AB85BC8556968C91B3
:100C70005697882309F111967C926E9213961C92D6
:100C80001E92129769857A85CD010E94B80000E016
:100C900024EF31E040E050E0B5018B859C850E9457
:100CA000A80081E0EB85FC85858387838CE090E05C
:100CB0009183808313821282AB85BC8512968D91BD
:100CC0009C911397019613969C938E931297D1CB78
:100CD000128613861486158616861786108A118A40
:100CE000128A138A148A158A168A178A2C960FB6C6
:100CF000F894DEBF0FBECDBFDF91CF910F91FF9073
:100D0000EF90DF90CF90BF90AF909F908F907F90AB
:100D10006F905F904F903F902F9008959C01245FBB
:100D20003F4F621773073CF048966817790718F42D
:100D300081E0FB0180830895FC0184810895FC011A
:100D400085810895FC0186810895FC0187810895BD
:100D5000FC0180850895FC018185089521E0FC0156
:100D60002287089521E0FC0123870895CF92DF9226
:100D7000EF92FF920F931F93CF93DF93EC01898142
:100D80000E949C098C018F8190E00817190731F0AF
:100D90000E94BD08688779878A879B870E94BD0863
:100DA000C884D984EA84FB846C197D098E099F0963
:100DB000CB80DC80ED80FE80C616D706E806F906FB
:100DC00078F4888190E00817190751F081E0011547
:100DD000110509F480E08883EC85FD85CE01099535
:100DE00081E0012B09F480E08F83DF91CF911F9187
:100DF0000F91FF90EF90DF90CF900895DF92EF92E8
:100E0000FF920F931F93CF93DF93EC01D62E7A01BD
:100E100069837A8302E310E020E030E00B831C83D7
:100E20002D833E83862F0E949C0921E0892B09F4A3
:100E300020E028831F82188619861A861B86FD8665
:100E4000EC8660E08D2DDF91CF911F910F91FF9087
:100E5000EF90DF900C942D094F925F926F927F92EA
:100E6000AF92BF92CF92DF92EF92FF920F931F93B8
:100E7000CF93CE2DDC014D905D906D907C90A12C98
:100E8000B12CC12CD12C7601C414D504E604F7048E
:100E900014F5DC011496ED91FC911597EA0DFB1DFC
:100EA000BFEFCB1ADB0AEB0AFB0AAFE0AA0EB11CBC
:100EB000A185B285AB2B41F752874187008311830F
:100EC00022833383C48374876387968785871582DB
:100ED000168217821086CF911F910F91FF90EF908D
:100EE000DF90CF90BF90AF907F906F905F904F90CA
:100EF0000895CF92DF92EF92FF920F931F93CF93BB
:100F0000DF936B01EC01088119812A813B81A0E00C
:100F1000B0E040E050E0BA014017510762077307A4
:100F20009CF4EC01EC81FD81EA0FFB1F4F5F5F4FEA
:100F30006F4F7F4F1F96E184F284EC14FD0461F73C
:100F40001286118614861386DF91CF911F910F911F
:100F5000FF90EF90DF90CF900895CF92DF92EF92C5
:100F6000FF920F931F93FC01DB0175836483208341
:100F7000318342835383C12CD12C7601C216D30610
:100F8000E406F50674F41A961C921E9219971E96A2
:100F9000FC93EE931D978FEFC81AD80AE80AF80A57
:100FA000EDCF178306831F910F91FF90EF90DF9095
:100FB000CF9008954F925F926F927F928F929F92FF
:100FC000AF92BF92CF92DF92EF92FF920F931F9357
:100FD000CF93DF93EC014A015B0100E010E0C12CEC
:100FE000D12C760188819981AA81BB81C816D90646
:100FF000EA06FB060CF056C0AC81BD81A00FB11F04
:1010000019966D917C911A976115710509F442C08A
:1010100015962D913D914D915C9118974D905D9055
:101020006D907C901397241535054605570594F56A
:10103000280D391D4A1D5B1D15962D933D934D932B
:101040005C93189724153505460557051CF11D9628
:10105000ED91FC911E970680F781E02D1B968D91F6
:101060009C911C970995EC81FD81E00FF11F848113
:10107000882381F085819681A781B0854081518147
:1010800062817381841B950BA60BB70B85839683B6
:10109000A783B0878FEFC81AD80AE80AF80A015F59
:1010A0001F4FA0CFDF91CF911F910F91FF90EF9035
:1010B000DF90CF90BF90AF909F908F907F906F9078
:1010C0005F904F90089508950E94C9080E94630898
:1010D0000E94BC00C0E0D0E00E94FC002097E1F339
:1010E0000E940000F9CF1F920F920FB60F921124A9
:1010F0002F933F938F939F93AF93BF9380917102F0
:1011000090917202A0917302B091740230917002BA
:1011100023E0230F2D3720F40196A11DB11D05C03A
:1011200026E8230F0296A11DB11D20937002809323
:10113000710290937202A0937302B0937402809133
:10114000750290917602A0917702B0917802019693
:10115000A11DB11D8093750290937602A093770232
:10116000B0937802BF91AF919F918F913F912F9152
:101170000F900FBE0F901F9018952FB7F8946091A5
:1011800071027091720280917302909174022FBF6C
:101190000895789484B5826084BD84B5816084BDEF
:1011A00085B5826085BD85B5816085BDEEE6F0E0E0
:1011B000808181608083E1E8F0E01082808182603C
:1011C0008083808181608083E0E8F0E080818160BD
:1011D0008083E1EBF0E0808184608083E0EBF0E0ED
:1011E000808181608083EAE7F0E080818460808391
:1011F000808182608083808181608083808180683B
:1012000080831092C1000895833081F028F48130EA
:1012100099F08230A1F008958730A9F08830B9F0B4
:101220008430D1F4809180008F7D03C08091800054
:101230008F7780938000089584B58F7702C084B53E
:101240008F7D84BD08958091B0008F7703C0809119
:10125000B0008F7D8093B0000895CF93DF9390E02E
:10126000FC01E254FF4F2491FC01EE52FF4F8491A8
:10127000882349F190E0880F991FFC01E650FF4F49
:10128000A591B49180519F4FFC01C591D4919FB716
:10129000611108C0F8948C91209582238C938881E9
:1012A00082230AC0623051F4F8948C91322F309529
:1012B00083238C938881822B888304C0F8948C913B
:1012C000822B8C939FBFDF91CF9108950F931F9333
:1012D000CF93DF931F92CDB7DEB7282F30E0F9010F
:1012E000E655FF4F8491F901E254FF4F1491F90143
:1012F000EE52FF4F04910023C9F0882321F0698347
:101300000E9404096981E02FF0E0EE0FFF1FE05119
:10131000FF4FA591B4919FB7F8948C91611103C0D0
:101320001095812301C0812B8C939FBF0F90DF917B
:10133000CF911F910F910895CF93DF93282F30E025
:10134000F901E655FF4F8491F901E254FF4FD49122
:10135000F901EE52FF4FC491CC2391F081110E940C
:101360000409EC2FF0E0EE0FFF1FEA51FF4FA591AB
:10137000B4912C912D2381E090E021F480E002C013
:1013800080E090E0DF91CF910895EE0FFF1F059070
:0A139000F491E02D0994F894FFCFCA
:00000001FF
